:020000040003F7
:10C0000060340020E1C20300F3C20300F5C2030064
:10C010000000000000000000000000000000000020
:10C02000000000000000000000000000F7C2030054
:10C030000000000000000000F9C20300FBC2030082
:10C04000FDC20300FDC20300FDC20300FDC20300E8
:10C05000FDC20300000000000DDE0300FDC203006E
:10C06000FDC20300FDC20300FDC20300FDC20300C8
:10C07000FDC20300FDC20300FDC20300FDC20300B8
:10C08000FDC20300BBD60300FDC20300FDC20300D6
:10C09000D1D60300FDC2030077E10300FDC2030017
:10C0A000FDC20300FDC2030000000000000000000C
:10C0B0000000000000000000000000000000000080
:10C0C00000F002F800F040F80CA030C8083824183E
:10C0D0002D18A246671EAB4654465D46AC4201D1C0
:10C0E00000F032F87E460F3E0FCCB64601263342B2
:10C0F00000D0FB1AA246AB46334318475439000020
:10C1000074390000103A02D378C878C1FAD85207BF
:10C1100001D330C830C101D504680C6070470000FD
:10C120000023002400250026103A01D378C1FBD853
:10C13000520700D330C100D50B6070471FB5C04611
:10C14000C0461FBD10B510BD03F010FC1146FFF72F
:10C15000F5FF00F01BF903F028FC03B4FFF7F2FF32
:10C1600003BC03F02DFC0000144C144D0646064F92
:10C17000F0B4034C024D024E014FF0B407480047A3
:10C18000000000000000000000000021000000008E
:10C19000000000000000000000000000F9FFFFFFA9
:10C1A000016881F308884068034AEFF305839A42E7
:10C1B000DAD1024CA646004700000000FFFFFFFF57
:10C1C000401E00BF00BF00BF00BF00BF00BF00BFD8
:10C1D00000BF00BF00BF00BF00BFF1D1704700002B
:10C1E000401E00BF00BF00BF00BF00BF00BF00BFB8
:10C1F00000BF00BF00BF00BF00BFF1D1704700000B
:10C2000070B505460C46164602E00FCC0FC5103E31
:10C21000102EFAD2082E02D303CC03C5083E042EFA
:10C2200007D301CC01C5361F03E021782970641CB7
:10C230006D1C761EF9D270BD2349224808607047F4
:10C2400010B500F01DF8002805D021491F484860AE
:10C25000C813204988612048018CC9B201290ED138
:10C26000818C09070BD1018D0906090F042906D11C
:10C27000808D0006000F02D118490120886010BD92
:10C280001548018CC9B2012917D1818C090714D135
:10C29000018D09060A0F03D1828D1206120F0ED0EE
:10C2A000090F012903D1828D1206120F07D003292D
:10C2B00003D1808D0006000F01D0002070470120BF
:10C2C000704700000024F40000200020DFFF07C0BA
:10C2D00000050040006C0040C00F00F00006004068
:10C2E0000A48026803210A43026009488047094856
:10C2F0000047FEE7FEE7FEE7FEE7FEE7FEE7000099
:10C3000005480649064A074B7047000024050040CF
:10C3100041C20300C1C00300602800206034002037
:10C32000602C0020602C002000F099F800F097F8B5
:10C3300010B502F095F810BD10B5644C86B01ECC57
:10C3400003946C460EC4002803D0684618DF00280A
:10C3500018D10F20800313DF002813D15C4B50222B
:10C360005C49092001F0DAFE00280BD169460490EF
:10C37000087404A860DF002804D1574801F0F3FED8
:10C38000002801D000F06BF806B010BD08B5534886
:10C39000C069B12822D0002451480F214069890387
:10C3A000884219D1012000070069012189028842D1
:10C3B00012D14C490320086001254B49A805C860EB
:10C3C00000F04CFA49480090494B05220321002017
:10C3D00001F0A4F9002803D000F041F80124DBE7C4
:10C3E00043490120143901F06BFD0028F4D13D4987
:10C3F00040484439086000F05CF900F0A1F90028D9
:10C400000ED000F0ACF90028E6D120466840FFF7D6
:10C4100093FF00F03CF800F0CBF90028DCD104E0F9
:10C420000120FFF789FF00F032F803252D03002CCF
:10C4300004D1A86800F08CF8002807D1FF203DDF68
:10C440000028C9D100F046F90028C5D1A86800F03D
:10C450007FF80028C0D0A86800F048F9BCE7BFF317
:10C460004F8F26492448C860BFF34F8FFEE71CB5A5
:10C4700001910090224A0821684601F0E1FB1CBDB1
:10C4800010B500211F4A084601F0DAFB10BD114A21
:10C4900010B550321421082001F0BEFB002801D055
:10C4A000FFF7DDFF10BD10B50246082901D0FFF7E8
:10C4B000D6FF11685068884710BD10B5002901D01B
:10C4C000FFF7CDFF01F0ECFD10BD0000E8F903001F
:10C4D00081C403005023002031C303000005004045
:10C4E0000010001058070050000500506FC40300F2
:10C4F00010210020040002000400FA0500ED00E015
:10C50000A7C40300BBC4030010B5C2480368012BD5
:10C5100002D1022900D10160100003D0BEA2432144
:10C52000FFF702FF10BD10B5BA4C40DF002803D062
:10C53000B9A25521FFF7F8FE01F0F5FB00F09AF9DA
:10C540002068022803D0032801D00428EDD110BDB3
:10C5500038B50068401C19D00024684600F078F90E
:10C5600000980168012910D1818800290AD0C1688A
:10C57000032000038068002201F06EFD0099898885
:10C58000814201D1012400E00024204638BD10B5CD
:10C590000446A0482021001D02F05BF9002803D0CA
:10C5A0009DA28C21FFF7C0FE9A480023202221463D
:10C5B000001D02F07AF8002803D097A29221FFF71D
:10C5C000B3FE10BD0FB438B5684600F041F900F075
:10C5D00051F96846818A049D97480122FF238D4CBA
:10C5E000002D1DD0012D21D0032D35D00021022D8D
:10C5F00041D0062D47D0FE23042D4ED0052D53D01B
:10C60000072D09D102F050FE002803D082A2F121AB
:10C61000FFF78AFE0420206038BC08BC04B018472D
:10C620008180089983600260C16010E08180079D6D
:10C6300006994919089D4919C160A52183600160C7
:10C64000069901610799856141610999C16122607B
:10C650007948FFF79CFFDFE700990B6803608B8840
:10C660008380C968C160AA21816006990161079928
:10C670004161089905E081800360C16001618360C8
:10C6800041618161E3E702F00FFE002803D062A25E
:10C69000D721FFF749FE0320BDE781800360C16019
:10C6A000009989688160D3E7036082808360C160FC
:10C6B000CEE70EB561480090202001900120029045
:10C6C00001F034FF002804D152496846091D01F0E9
:10C6D00056FF0EBD10B500F0CAF9002805D102F0D2
:10C6E0004FFF0446FFF71FFF204610BD70B511DF56
:10C6F000002804D0FF2148A23F31FFF715FE504922
:10C7000000200B684E4C012180340A4682401A42B8
:10C7100004D0C506ED0E0A46AA402260401C20281F
:10C72000F3D303242403A06813DF002804D0FF21DF
:10C7300039A24431FFF7F8FDA06800F085F870BD1C
:10C7400008B5684600F084F800980168A52904D06F
:10C750008068AA2801D0002008BD012008BD10B5BE
:10C7600000F09AFB002803D100F076FB00281ED0D1
:10C77000642002F03BF900F015FB002804D0FF21F3
:10C7800025A26931FFF7D0FD00F086FB002804D018
:10C79000FF2121A26C31FFF7C7FD00F03DFB040033
:10C7A00004D0FF211CA26F31FFF7BEFD204610BD53
:10C7B00000B589B01822234902A8FFF721FD069889
:10C7C00007990090019102A80FC8FFF7FBFEFFF741
:10C7D000AAFE002009B000BD10B50E4988B004467D
:10C7E00000232022091D684601F0E5FF0098206023
:10C7F00068468088A0800398E0600298A060049852
:10C800002061059860610698A0610798E06108B012
:10C8100010BD0000042000202E2E5C626F6F746C2F
:10C820006F616465725F6466755C626F6F746C6F74
:10C83000616465722E630000F024002009C50300C6
:10C8400000E100E0F8F9030010B5FFF7A9FC10BD06
:10C85000014901607047000000FC03000748012106
:10C86000C1600F225204426082680A438260044819
:10C8700001607047044903480860704700050140A3
:10C88000000001403546526E0006014070B5F94D7A
:10C890001E46AB6988B01446002B22D0284680681B
:10C8A000022902D004291CD105E0052819D13246FD
:10C8B0002146032014E0022813D11822EE4902A8D1
:10C8C000FFF79EFC069807990090019102A80FC8F7
:10C8D000FFF778FE0320A860AB69324621460220AC
:10C8E0009847200003D0E5A25E21FFF71DFD08B0A8
:10C8F00070BD4CB5DF4E01203070062001950094CC
:10C90000FFF760FE4CBD10B5DA4C2078002801D04E
:10C91000082010BD206901F005F8002803D0D7A237
:10C920008121FFF701FD0F2100228904206900F019
:10C930008FFF040003D0D1A28421FFF7F5FC20462D
:10C9400010BDCC4910B5CB48243141610221816032
:10C95000C168243002F013F8002803D0C7A29A213E
:10C96000FFF7E2FC10BDC349C2481C3141610321FD
:10C9700081608369002B03D00022114602201847F2
:10C980007047C74900204A680321090389688A4221
:10C9900008D9511A880A80028905890D02D001211F
:10C9A00089024018704700B5B24987B049886A4685
:10C9B00011810321090389680691B94901204A6858
:10C9C00003928A680492C9680591069A00910192BF
:10C9D00002A90EC9FFF7F6FD002007B000BD30B573
:10C9E000AF4CA44887B02430E16801F0C8FF0028AC
:10C9F00003D0A2A2F421FFF797FC9E48E2681C3006
:10CA000041680023083001F08AFF0546FFF732FF36
:10CA1000002D07D0042001960094FFF7D3FD28468F
:10CA200007B030BD00209349019049886A461181C2
:10CA3000E1680591069A0091019202A90EC9ECE7FE
:10CA400000B58C4987B049886A4611819449032012
:10CA50004A6803928A680492C9680591069A00910F
:10CA6000019202A90EC9FFF7ADFD0020B5E7F0B5B0
:10CA7000814A91B0183207CA02AB07C303263603B6
:10CA8000B0680F218903091A7A4C49084718002514
:10CA9000657021466580243102A801F024FF00283A
:10CAA00023D121462431B068486024390A46526AAD
:10CAB000CA610F218903091A4908401821461C310F
:10CAC000486005A8FFF788FE0798FE2802D138685D
:10CAD000401C12D00F20B1688003401A41086548FD
:10CAE0001C3001F04CFF002802D0A56011B0F0BD51
:10CAF0000DA90EC90520FFF765FD5E48694A0021B2
:10CB0000103000F05EFE002804D0FF215BA25531FA
:10CB1000FFF70AFC0F2100228904206900F098FE2B
:10CB2000002804D0FF2155A25931FFF7FDFB012059
:10CB30006560A0600020D9E74E498861704770B5F4
:10CB400042685748146853689168D268046043602B
:10CB5000C26081600078440701D5840705D19C0735
:10CB600003D18C0701D1940701D0062070BD5B185A
:10CB70009A18404D0F239B02EA60994214D84A4903
:10CB80004A4CC30709D08868EF218902081A9042ED
:10CB90000AD34748206047480FE089680F239B036A
:10CBA000591A4908914201D20C2070BD42492160B6
:10CBB000800701D5414800E041486060A86801282D
:10CBC00002D00826304670BDFFF79DFE0600FAD160
:10CBD0002168E8688847F5E770B5050004D0287A31
:10CBE000800703D0102070BD0E2070BD214CA068BE
:10CBF000032805D0042803D0052803D0082070BDE1
:10CC00000520A0606868E168860060688019884235
:10CC100004D90020C04360600C2070BDFFF773FE94
:10CC20000028FAD1A96832466368606901F077FE8E
:10CC30000028F2D1616889196160E2689142ECD004
:10CC4000092070BDF8B50B4C0546A068032802D03A
:10CC5000042805D101E00420A0606068002801D00C
:10CC60000820F8BDFFF74FFE0028FAD10C4B002139
:10CC7000103330E01020002010FA03002E2E5C62EA
:10CC80006F6F746C6F616465725F6466755C646617
:10CC9000755F6475616C5F62616E6B2E630000008E
:10CCA00010250020F3C80300003000003C200020C5
:10CCB00043C90300A7C9030067C9030041CA0300B1
:10CCC000DFC90300AA688E00965962789700521C4B
:10CCD000DE516270491C6A688A42F3D8F8BD70B5AB
:10CCE0008E4CA068052805D10620A060E168606828
:10CCF000884201D0082515E0FFF705FE050011D197
:10CD0000606900224068E16801F0A6F9608084490A
:10CD100062780988002A03D0884201D00B2070BDB8
:10CD20000720A060284670BD10B57C48816807299F
:10CD300001D0082010BD006900F0F4FD002803D0E8
:10CD4000784A7949FFF7F0FA74482C3040688047F8
:10CD500010BD1CB5072001950094FFF733FC1CBDE6
:10CD6000F8B51C4617460D46064600F0C1F80028E7
:10CD700017D001200003854207D92346291B301B09
:10CD80001A46FFF7EDFF00280BD13A4629463046F8
:10CD900000F0B9F8002804D13A462946304600F0A0
:10CDA000A7F8F8BDF0B589B06846FFF715FD0498FF
:10CDB00000282AD001210903079A4018904226D959
:10CDC000501A45081046049A0C4687180246680017
:10CDD00016180019089003200003806804998842FF
:10CDE0000DD261190846042200F08DF800280CD1FC
:10CDF00021460422084600F086F8002805D1BA1B17
:10CE00002B4630460899FFF7ABFF09B0F0BD049AF6
:10CE1000079800F078F8F8E700B58DB004A8FFF7A0
:10CE2000DBFC099800280DD0089800280CD0089940
:10CE30000B984018019000210998009180080290F9
:10CE4000684618DF0DB000BD0320000380680F2185
:10CE50008903091A4908ECE700B58DB004A8FFF76B
:10CE6000BBFC09980028EDD00F2108988903002801
:10CE70000CD0089A0B98019180180290032209980F
:10CE8000009280080390684618DFDBE70320000368
:10CE900080680A1A5208EEE730B591B06846FFF78D
:10CEA0009BFC0498002814D001210903079A40181C
:10CEB000904214D9501A43081046049A5C00821814
:10CEC0000019611803242403A468049DAC4202D213
:10CED0000E2011B030BD121AFFF742FFF9E7032010
:10CEE0000CAB07C3049880080F900CA818DFF0E77C
:10CEF0001FB50323019090080390009302916846A8
:10CF000018DF04B010BD1FB50123019090080390F5
:10CF100000930291684618DFF3E70000102000201C
:10CF2000202500207CCC03007202000030B585B0C3
:10CF3000002822D00388FA4CA34220D0F94B1B785A
:10CF4000002B1CD0F74B10255B1C1D705970002462
:10CF500001259A70032269460A8200940194029482
:10CF60000394C2890A808D708C8004A90291039376
:10CF700000886946A6DF05B030BD0E20FBE708201B
:10CF8000F9E7F0B589B004460227684607700D46F8
:10CF90008783608A08AB07AA0021A5DF0026002846
:10CFA00004D0616A00291AD0884718E06846008CCE
:10CFB000C007C00F13D06846868020886946A8DF66
:10CFC000002812D1A97E284601221B300B0002F056
:10CFD000FEFC093F0E1E202224263D283F00FF2094
:10CFE000FE30694688802088A8DF09B0F0BD04962D
:10CFF000298B022902D26846067502E069460A7545
:10D000000690226A04A9204690470020EDE704928A
:10D01000F7E70497F5E7032014E0042012E0052069
:10D0200010E0298B032905D2032208212046FFF7AF
:10D030007DFFDAE74178027808021043694688826A
:10D0400002D006200490DCE70720FBE70920F9E77F
:10D050000322EBE730B585B00D46040032D0002D39
:10D0600030D0286800282DD00020C043AE4B20804F
:10D070000FCB049301AB07C3AC4869460880891CF9
:10D0800001A863DF00281CD1A21C69460120A0DF93
:10D09000002816D1684680782071204600F0C0F83C
:10D0A00000280ED1204600F0F9F8002809D12868A0
:10D0B00020626868002800D060629A4901200870E8
:10D0C000002058E70E2056E73EB5002820D0002962
:10D0D0001ED0026A002A1BD00A88102A19D0112AF1
:10D0E00028D0502A17D0512A12D10446891D087819
:10D0F00002280DD14888E289904209D1891C204636
:10D10000FFF73FFF002803D0616A002900D088475D
:10D110003EBD898810E0CA88C3889A42F8D10822A7
:10D1200000928A7F6B461A7120310291026A694629
:10D1300090473EBD0021C94301803EBDF0B585B09A
:10D140000A4605002DD02888754988422BD075489D
:10D150000078002827D0734C1020641C2070072012
:10D1600060700127A7700321684601820026E11C38
:10D17000104600F04CF801466846008A09186846D7
:10D1800001820096019602960396E98901808770D4
:10D19000868004A80394029028886946A6DF05B01B
:10D1A000F0BD0E20FBE70820F9E7F0B585B00A4690
:10D1B000050028D028885A49884226D05948007846
:10D1C000002822D0574C1120641C2070012768468B
:10D1D00007820026611C104600F019F801466846D7
:10D1E000008A091868460182009601960296039605
:10D1F000E98901808770868004A8039402902888BA
:10D200006946A6DFCBE70E20C9E70820C7E708700C
:10D21000020A4A70020C8A70000EC870042070471F
:10D2200030B58FB005461C21684602F0DCFA69462D
:10D230000878042108436946087000240194039487
:10D24000049405940694287908A98870374869469B
:10D25000801C0884601C00070794000F0C771030B6
:10D2600048778A7FF9200240921CE7200240012083
:10D2700002438A77142109A802F0B5FA08A8099098
:10D2800007A80A9069468C851420CC8508860D94E1
:10D290006888AB1D09AAA2DF0FB030BD30B58FB0D2
:10D2A00005461C21684602F09EFA69460878082166
:10D2B0000843102210436946087000240194039427
:10D2C000049405940694287908A98870174869463B
:10D2D000401C0884601C00070794000F0C77103076
:10D2E0004877887FF9210840801CF72108401043C7
:10D2F0000121084369468877142109A802F073FACE
:10D3000008A8099007A80A9069468C851720CC8543
:10D3100008860D942B4668880E3309AAA2DFBBE766
:10D32000FFFF00004420002034FA03003015000005
:10D330005748002101705848564A02608160C16018
:10D340000161082241614260816108467047002006
:10D350007047002805D04E490A78002A03D00420DF
:10D3600070470E20704701220A704949491C01602C
:10D3700000207047464900200870704710B500290A
:10D380001DD000220A60444A5368002B1BD020287D
:10D3900017D85B1E5360D0682423401CD0601069EE
:10D3A00014684343E3180B60012383409169401CD8
:10D3B00019434007400F91611061002010BD0E20FD
:10D3C00010BD0C2010BD042010BDF0B5324A064639
:10D3D000916800292BD057691020791A4907490F05
:10D3E00014680B4624254D436519B54206D1012426
:10D3F00095698C4065400020956104E0491C49070F
:10D40000490F8F42EED1491C4E07760F95690121D5
:10D410000C469C402B4623420AD19368002B07D030
:10D420005B1E936053685B1C53603346F0E7042037
:10D43000F0BD194A2423117C1268491E4907490F7F
:10D440005943203150500020704770B500281AD041
:10D45000002918D0104AD368002B16D05B1ED36069
:10D46000936824265B1C9360536915681C467343BC
:10D47000EE1820330660E858641C08606007400F0F
:10D480005061002070BD0E2070BD042070BD0000F2
:10D490004C20002060250020802600208307FF22EA
:10D4A000DB0E9A408907090E994000280BDA000725
:10D4B000000F08388308FF489B001B18D869904369
:10D4C0000843D86170478308FB489B001B18186805
:10D4D000904308431860704770B50124F749600411
:10D4E0000860F74940108860F54940398860F54D7B
:10D4F0006C602F20FEF764FEAC60F34D00242F20FB
:10D500006C61FEF75DFE2C7170BDF0B5EE4F282109
:10D51000BC6841430D1939694A1C09D028224A4385
:10D520001619AB68B268934204D8D21AB260696225
:10D530003861F0BD0A4602E00A46796A9B1B4E1C20
:10D540000BD028264E433719BE689E42F4D32826B6
:10D550004E433619B768FF1AB760AB60696228217D
:10D560004A4311194862F0BDF8B5D74C2569681CCB
:10D5700036D0D648002640686169401A07023F0A43
:10D580001AE028204543A0682A189068B84215D8A8
:10D59000A3693F1A8619556A002B0AD0116AD0690F
:10D5A0009847002808D0FF21C9A26331FEF7BCFECE
:10D5B00002E0D169106A8847681CE2D1A178E0785E
:10D5C000814206D1401CC0B2E070022801D1002087
:10D5D000E070BD490006800D1C310E5000F0F4F9DA
:10D5E000F8BDF8B50446B84801690091467856E0A0
:10D5F000B548F100C2688D184BE0601C07D0B24AF4
:10D60000282192686143204689184C6A20E02878D6
:10D61000182141436A68401CC0B252182870A9788A
:10D62000884201D100202870A74B506828219B68B0
:10D630004143C9181368012B2DD10B7E002B2AD131
:10D640009368CB60D3680B6113694B6152690A62BE
:10D650009D4ACF685369BC46FA1A1202A84F120AB3
:10D66000BA4202D20B69D21809E062469A1A120233
:10D670000B69120A934201D99A1A00E000228A60CB
:10D680000022CA600A6101220A76921E4A62FFF7EE
:10D690003CFF601CB1D1287869788842ADD1304612
:10D6A000761EF6B20028A3D187480169009881420E
:10D6B00001D00120F8BD0020F8BD9249002008608B
:10D6C00048608860C8608F494039086048604BE70F
:10D6D000F0B5002087B0C04302907B4846690569D9
:10D6E000684600F076F9074600F090F90446002FEE
:10D6F00008D002AA3146009800F0D0F90298FFF74E
:10D7000070FF06E00298FFF76CFF002801D1002CA3
:10D7100002D0284600F0EBF907B0F0BDFFB598073E
:10D72000002481B01E4615460F4600280BD1002E5E
:10D7300009D0FFF7D1FE64490A9888610F7032461C
:10D7400000208E6008E0072005B0F0BD2823434389
:10D75000D4509B181C76401CB842F7DB2820474366
:10D76000BB19032048700F461846CB601946183085
:10D77000002218232E465E43D3005B181C705C7099
:10D780009D7058603018521C032AF5DB0020C043FE
:10D790003861BC70FC7001245B48240504600321DF
:10D7A0001420FFF77BFE454880380460474C019801
:10D7B000A06003211120FFF771FE606878610020EE
:10D7C000C2E770B5404CA568002D06D0002A06D0EF
:10D7D000002804D00023247809E0082070BD072029
:10D7E00070BD28265E43AE59002E04D05B1CA342B8
:10D7F000F7DB042070BD282401265C432E516419F8
:10D80000E26161600360002070BD2A494868C0057C
:10D81000C00D17D0103807D50207120F083A92082A
:10D8200092005118C96904E08108234A89008918C7
:10D8300009688007C00EC1400806800F012803D088
:10D84000032803D002207047002070470120704752
:10D85000FEB504461C48174682680D46002A0CD0C7
:10D8600001788C4201D2052D01D20720FEBD214650
:10D87000282359435358012B01D00820FEBD881896
:10D88000406801284AD00026FFF7BFFFC0000E49BC
:10D890000190C9684018694600F06FF900283FD030
:10D8A000012144600160094949680830E2C0064925
:10D8B00001982BE000ED00E000E400E080E100E0F2
:10D8C0004013014000100140542000200015014089
:10D8D0002E2E5C2E2E5C2E2E5C2E2E5C2E2E5C535D
:10D8E0006F757263655C6170705F636F6D6D6F6E95
:10D8F0005C6170705F74696D65722E63000000007A
:10D90000FFFF7F004011014080E200E0C96841183C
:10D910000098487000F058F80020FEBD2E46B3E78E
:10D920000420FEBDF8B5B64D0446A868002809D00D
:10D9300029788C4201D30720F8BD28216143405843
:10D94000012801D00820F8BDFFF75FFFC600E86896
:10D950006946301800F011F9002809D0022112C0E0
:10D96000E86831180098487000F02EF80020F8BDE3
:10D970000420F8BD38B5A24CA068002815D0FFF7E8
:10D9800044FFC500E0686946281800F0F6F8002852
:10D990000DD003210160091F4160E068291800983B
:10D9A000487000F011F8002038BD082038BD042070
:10D9B00038BD94494968016000207047401A000250
:10D9C000000A10600020704701208F4900050860A0
:10D9D000704710B58A4900238A78CC78A24212D0C9
:10D9E000521CD2B28A70022A00D18B708A78844B82
:10D9F00092001C339A580260486910180002000A0D
:10DA00004861012010BD0360002010BDF8B57C48BE
:10DA100001690091457833E07948E900C0680E1843
:10DA200034782AE0182060437168641C0818B178C3
:10DA3000E4B2A14200D100240168022902D00329E6
:10DA40001BD113E06E4A40682821926841438F1829
:10DA5000397E002911D000F0A2F8002038760CE0C1
:10DA600028277843C0180276406A03E06449002200
:10DA70008B680869471CF3D108617078A042D1D146
:10DA800028466D1EEDB20028C6D15D480169009898
:10DA9000814201D00120F8BD0020F8BDF7B5584CF7
:10DAA0000025A76823691EE028215943C9198E68FB
:10DAB000864202D9301A886017E0801B751900264B
:10DAC0008E600E764E699C464B6AB646002E0AD092
:10DAD000019E76193602360ACE6076460E611668C9
:10DAE0004E6261461160591CDED12361FEBDF8B55E
:10DAF000434801694A1C3DD0282251438268891855
:10DB00008E6840494C6847690079E11B0D022D0A77
:10DB1000ED1C002815D101203C4A000450603B4A0E
:10DB2000403A506038494000803108603849086008
:10DB30003849012008602F20FEF742FB30490120C0
:10DB40000871B54200D23546E81900022D49000A95
:10DB5000403108602B494968001B091B0902090A6A
:10DB60000002C91C000A814203D901202649400451
:10DB70000860F8BDFFF7B0FCF8BD42788378521C0E
:10DB8000934200D100220378934201D100207047D4
:10DB90000A6041684078182250430818704770B5F1
:10DBA000174E3569B26829460C4606E0844207D014
:10DBB000254628235C43A3185C6A631CF6D170BD1C
:10DBC000002BFCD0A54208D1282041438818406A88
:10DBD0003061401C01D1FFF77FFCB168282044432D
:10DBE0006018282382685D43406A6B185862431CA2
:10DBF000E5D028235843401881688918816070BD9A
:10DC0000542000200015014000E200E040130140D4
:10DC100000E100E00010014030B5CB0008339DB2B8
:10DC200093070024002B01D0072030BD554B9A608C
:10DC30005219DA605C701C7058809980002030BDE9
:10DC4000F7B5504C82B060880F4681426AD80020F8
:10DC5000694608704D494C4E4868C005C00D16D045
:10DC6000103807D50207120F083A9208920051188F
:10DC7000C96904E08108464A890089180968800753
:10DC8000C00EC1400806850F012D01D10AE0042510
:10DC900068462EDF02280BD0002803D03DA2592170
:10DCA000FEF742FB6078A188884203D2401C02E064
:10DCB00072B6F7E700202278C0B2904207D06678AB
:10DCC0006078884201DA401C00E000206070012D7D
:10DCD0000BD062B6684600782FDF022805D00028F6
:10DCE00003D02CA26121FEF71FFB2748864219D0E2
:10DCF000A068F50004994151029900290CD0002F29
:10DD00000AD060883A464643E068301801F00CFDBE
:10DD1000A0682818878002E0002128188180002050
:10DD200005B0F0BDFEE70EB504E068468188029AB2
:10DD30000098904702AA01A9684600F003F800285D
:10DD4000F3D00EBD70B50F4B05245D781E78B5423B
:10DD500015D01D781C789E88B44201DA641C00E05E
:10DD600000241C705C88DE686C43A41904609B6806
:10DD7000E800C418A4880C801858002410602046BD
:10DD800070BD000078200020FFFF000000ED00E0E3
:10DD900000E400E02E2E5C2E2E5C2E2E5C2E2E5CDF
:10DDA0002E2E5C536F757263655C6170705F636F7C
:10DDB0006D6D6F6E5C6170705F7363686564756CC8
:10DDC00065722E6300000000F0B5002201230326D7
:10DDD00036041F4697400C463C420FD0C5682C467F
:10DDE0003C420FD03446BD43C560934D97007D192A
:10DDF0002F68B7432F602F6827432F60521C202ABB
:10DE0000E7D3F0BD012464043D43EDE7F8B58B484A
:10DE100005698B490020C863074632E014213A4661
:10DE20004A434168806854180121B940014226D014
:10DE3000E068C64320686E40064031462046FFF742
:10DE4000C3FF7E48006968400CD00543E068216844
:10DE5000C04368400840014600902046FFF7B4FFE9
:10DE6000009806433046A168A84301402A466068EE
:10DE70003240104002460A4301D0226990477F1C7D
:10DE8000FFB2704841788F42C8D3F8BDF0B56D4AF3
:10DE900000215368142250430124674D03273F0497
:10DEA0001E5822468A40164206D08A005219166829
:10DEB000BE43166016681660491C2029F0D3F0BDD9
:10DEC00010B5002903D08A070024002A01D00720BA
:10DED00010BD5C4A0B4651601070142154704143D0
:10DEE0001846946001F07FFC00205749C0438860C9
:10DEF000564840210160564A1068FF231B0498438E
:10DF00000B041843106053480160002010BDF8B5A1
:10DF10004C4F84467D68002D07D0002B07D07878C1
:10DF20003C78A04205D30420F8BD0820F8BD0720A6
:10DF3000F8BD0E461424164344432E516419236140
:10DF4000A260616061460870411C7970FFF79EFF16
:10DF50000020F8BDF0B53B4A5168002904D0537841
:10DF6000984203D30720F0BD0820F0BD344B0025B4
:10DF7000DD63324B1C699768002F02D1324EDB05FE
:10DF80007360012686403E43966014225043421837
:10DF9000D560002201230D5893401D4216D025461E
:10DFA0001D4202D003252D0405E001256D0446180D
:10DFB000F7681F43F760204B9600F3181E6803278D
:10DFC0003F04BE431E601E682E431E60521C202A62
:10DFD000E0D30020F0BD70B51A4C054660680028FB
:10DFE00004D06078854203D3072070BD082070BD3F
:10DFF0002846FFF74BFF0121A068A9408843A06095
:10E0000003D101201049C0078860002070BD0D4B6E
:10E010005A68002A04D05B78984203D307207047DF
:10E0200008207047142358438018044A1269006876
:10E03000024000200A6070470007005000050050B1
:10E0400040610040882000200063004080E200E042
:10E0500004E400E000E100E010B50446002A02D02C
:10E060001088002210E00A48FBE7030A000203437D
:10E07000A05C584003061B0F43401803584083B26E
:10E080001806C00C5840521C8A42EED310BD000046
:10E09000FFFF000010B508461146FEF747F910BD16
:10E0A000F8B53D4C2078002837D02069002807D0EB
:10E0B0000026E068002805D00025002E04D013E0DB
:10E0C0000126F6E70125F8E7684651DF052806D066
:10E0D000002806D031A26921FEF726F904E00126C6
:10E0E00002E0216900988847002D12D160886946B6
:10E0F0000880A06861DF052806D0002806D027A286
:10E100008021FEF711F904E0012502E0E168A06832
:10E110008847002ED8D0002DCFD0F8BD70B500298B
:10E1200001D08C0701D0072070BD1B4C0125A160D8
:10E1300062802849636010DF0028F5D12570162021
:10E1400026DF70BD11DF002801D0012100E0002191
:10E15000114A11707047002803D00F49C860002091
:10E1600070470E207047002803D00B49086100203B
:10E1700070470E20704710B507484068002808D047
:10E180008047002804D0FF2104A23331FEF7CCF8E9
:10E1900010BDFFF785FF10BD942000202E2E5C2EB1
:10E1A0002E5C2E2E5C2E2E5C2E2E5C536F757263B1
:10E1B000655C73645F636F6D6D6F6E5C736F6674C7
:10E1C0006465766963655F68616E646C65722E6311
:10E1D0000000000095E0030018225043FE4A002191
:10E1E0008018017181604161012281610261C16019
:10E1F0007047FFB581B0F94C049B039A0546266928
:10E200001A4303200092002E03D1002A0ED00122CF
:10E2100022612769039A0126360792003B0001F02C
:10E22000D6FB072707162940526127000222EFE795
:10E230007069326992B25043326933691204920CA8
:10E240009BB2594321DF002812D102210FE008467A
:10E2500020DF00280CD10399002901D0032106E01A
:10E260000499002916D12978042946D017E02161A4
:10E2700005B0F0BD7069326992B25043326993B211
:10E280004B4301461846039A21DF0028F0D1049938
:10E29000002901D00421EAE72978042920D00521AA
:10E2A000E5E773693069366980B2434368681B18D3
:10E2B0009B18B6B24E43301880181946049A21DFD5
:10E2C0000028E9D0D4E7306980B2484369688018F3
:10E2D0008A08696921DF0028CAD1009900290CD079
:10E2E0000621C4E77069316989B24843316989B24E
:10E2F00001F08CFA20DF0028BAD10721B7E7F8B582
:10E30000B54918230A780F205A435418241DB349DD
:10E3100022782669CF68022A1BD001252D07042AFE
:10E320002AD0052A5BD1286981B2304601F06EFA05
:10E330000146A36828699A1980B24843101A8208D6
:10E3400060681818861928694B1C80B25843801BD6
:10E3500034E0B80262686169121A0918A3683018BB
:10E36000181801239B029A4202D2920821DF31E061
:10E37000FF22013221DF2DE0E2689749142050434B
:10E38000F4314018001D0BC8B04203D160685943F6
:10E39000814218D0022A16D0286981B2304601F095
:10E3A00035FA0146286980B24843301A8208286944
:10E3B0004B1C80B2584363689B19C01A83082046DF
:10E3C000FFF717FF06E0286981B2304601F01EFA18
:10E3D000C01920DF002802D17F4901228A70F8BDD0
:10E3E000F8B57D4C069E65780A2D1DD027787D19DD
:10E3F000EDB20A2D01D30A3DEDB218277D432D1948
:10E400002871AA6103C9EE60AB6069612861A178D7
:10E410000020002904D1FFF772FF112800D100204D
:10E420006178491C6170F8BD0420F8BD38B502461A
:10E430006948182301785943081803690179022BA8
:10E440000AD014246343644CF434E4588368009382
:10E4500083691030A04738BD604B14331C68F5E762
:10E46000F8B55D4B9978012914D100255B499D7061
:10E470000A69082A05D002280FD003280AD10D20E6
:10E4800006E0022807D00D7000F09DFA002801D0A8
:10E49000FFF7CCFFF8BD0D61F6E74F48182403786D
:10E4A0004E496343CC681818641C001DCC60037887
:10E4B000022B05D14668A102B14201D3012700E039
:10E4C0000027052B01D1072A03D00021042B02D0FD
:10E4D00003E00121FAE7072A03D00026042B02D02B
:10E4E00007E00126FAE74068A302834201D3002A2D
:10E4F0001AD00020314301433943C5D0374E284656
:10E500003561FFF793FF344C2078FFF765FEF56027
:10E510006078401E60702078401CC0B220700A28CD
:10E52000B2D30A382070AFE70120E3E770B50025C9
:10E530002A4C2948E56025610570457085702E4696
:10E540003046FFF749FE761C0A2EF9D30122120746
:10E550006560516928461269491E92B25143E560CF
:10E56000A1601D49F4310D608D600D61CD601B49C6
:10E5700014310D60888001212170206170BDF8B5D3
:10E58000164A044610780E46002830D0002C30D0B1
:10E59000002E2ED0206800282BD0012000076768AD
:10E5A000016989B28F4228D8102F26D3A16800298B
:10E5B00023D09568794343694A19006980B243437F
:10E5C0009A421AD801200007006980B2814212D90C
:10E5D00001200007006903E09C260020A8200020FD
:10E5E00080B2394601F012F9002906D103E0082073
:10E5F000F8BD0E20F8BDB80701D00720F8BDF949D5
:10E60000486801281CD00F461421F74A21C641430F
:10E610008E187560236853506168B160A168F1601D
:10E62000A268616800235143012212075B1C146930
:10E630009BB2A4B28C4205D21469A4B2091B02E0B9
:10E640000420F8BD00211469A4B265191469A4B2AC
:10E650008C42EBD9BD60401C336178600020F8BD6E
:10E6600030B5E04B1B78002B07D0002807D0002ADC
:10E6700005D00468002C12D103E0082030BD0E2024
:10E6800030BDD94B1D68002D09D0456898684143BD
:10E690006918DD68454358682818884201D8072062
:10E6A00030BD14600020516030BDF8B50446CD483F
:10E6B0001E46007815460F46002807D0002F07D0C9
:10E6C000002C05D02068002817D103E00820F8BDF1
:10E6D0000E20F8BDC448016800290ED0C2688168C8
:10E6E00040684A4310186268904206D9002D04D051
:10E6F000A94202D3A819884201D90720F8BD38469B
:10E7000000F05BF9002811D0304600F056F90028DF
:10E710000CD0606800F051F9002807D02B463A462B
:10E72000214602200096FFF75BFEF8BD1020F8BDE1
:10E73000F8B50446AB481E46007815460F4600283B
:10E7400007D0002F07D0002C05D02068002817D153
:10E7500003E00820F8BD0E20F8BDA3480168002999
:10E760000ED0C268816840684A43101862689042BF
:10E7700006D9002D04D0A94202D3A819884201D994
:10E780000720F8BD384600F018F9002811D03046AF
:10E7900000F013F900280CD0606800F00EF9002892
:10E7A00007D02B463A46214605200096FFF718FE73
:10E7B000F8BD1020F8BDFFB58A4881B000781F462B
:10E7C00016460D46002808D0002D08D001980028D4
:10E7D00005D02868002817D103E0082048E50E205E
:10E7E00046E5814C206800280ED0E168A068626888
:10E7F000414389186A68914206D9002E04D0B0427C
:10E8000002D3F119814201D9072031E5019800F0C6
:10E81000D4F800281BD0384600F0CFF8002816D0D6
:10E82000686800F0CAF8002811D068683246C1193B
:10E83000019800F079FF0096286814214843245875
:10E84000002203212846019BA047002010E510204C
:10E850000EE5F8B5054663480F460078002805D058
:10E86000002D05D02868002821D103E00820F8BD3C
:10E870000E20F8BD5C4C00262068002817D0A16847
:10E88000E068484361684118686881420FD900F028
:10E8900094F800280DD0296814225143091968689A
:10E8A0004A688968801A00F0B1FF002903D0072068
:10E8B000F8BD1020F8BD3B460022294604200096F2
:10E8C000FFF78EFDF8BD47490978002907D00028D9
:10E8D00007D04549F4394978016000207047082085
:10E8E00070470E2070473F4A1278002A0DD000284A
:10E8F0000DD000290BD00268002A08D0394A143202
:10E900001368002B05D004207047082070470E20A4
:10E91000704702230B600068106000207047F8B554
:10E92000044630481E46007817460D46002807D09A
:10E93000002D07D0002C05D0206802281BD103E051
:10E940000820F8BD0E20F8BD2648143000680028C5
:10E9500011D0084600F031F800280ED0304600F003
:10E960002CF8002809D03B462A4621460220009672
:10E97000FFF736FDF8BD0720F8BD1020F8BD08B53B
:10E98000184A1278002A05D0002805D00268022A09
:10E9900011D103E0082008BD0E2008BD114A143231
:10E9A0001268002A07D00B4600220146042000927C
:10E9B000FFF716FD08BD072008BD800701D0002025
:10E9C000704701207047084910B5F4394978002094
:10E9D000002906D0FFF793FC002802D0112800D1AF
:10E9E000002010BDA82000209027002031B5054C44
:10E9F00004E0401E00902046FDF7F2FB009800283E
:10EA0000F7D138BDE703000038B57A497A4A48881B
:10EA100090420FD04A78794C521CD2B24A70237B74
:10EA2000934208D3083175DF002803D0A16900297B
:10EA300000D0884738BD00254D70217C002907D0C3
:10EA40003B2176DF002803D0A169002900D0884748
:10EA500061690029EED068460095884738BD70B5D9
:10EA6000054601461C226548FDF7CAFB614C00269D
:10EA700026702968002907D00822A01800F054FE4B
:10EA8000204608307ADF02E05A4808307BDF002851
:10EA900008D1401E608057486670594A0021001D09
:10EAA000FEF78FFE70BD10B552484068FEF73AFF82
:10EAB00010BDF8B54F48103000F08EF800264D4DCF
:10EAC0004E4C002806D06169002919D00120009021
:10EAD000684614E02878002804D0616900290FD026
:10EAE0000096F5E7687800280CD0A16800226868D5
:10EAF000FEF7AEFE002803D0A169002900D08847A8
:10EB00002E70F8BD6168F1E7F8B53C4C028800272B
:10EB1000384DE689102A18D029464968112A21D093
:10EB2000122A2DD0502A0FD1801D0288B2420BD15B
:10EB3000028B022A08D1C27E837E10021843C007CE
:10EB4000C00F13D0FFF7B5FFF8BD8188698001467B
:10EB5000284808220E31103000F0E6FD6F70002EBC
:10EB6000F0D0F8BD0020C04368806F700846FEF703
:10EB7000D9FE0028F5D0A1690029F2D08847F8BD58
:10EB8000811D1C480822103000F0CEFDDAE7F8B5F0
:10EB9000014618480822083000F0C6FD1548083024
:10EBA0007ADF04000DD11348103000F015F801256C
:10EBB000002808D011484169002902D06846009514
:10EBC00088472046F8BD0B4E3570314608317088B5
:10EBD00075DF04467570F4E74188064808300288FE
:10EBE000914204D34088814201D80120704700201F
:10EBF00070470000C4200020FFFF0000A427002071
:10EC000009EA0300FFB583B0074600200C9C864646
:10EC1000267805463AE07868A90041180A886846CF
:10EC200082804988C1800022694601A865DF0028EA
:10EC300010D1684601780598814226D17046002897
:10EC400001D0002200E002222078891841181F29F3
:10EC500002D90C2007B0F0BD7146002908D1401C34
:10EC6000C0B2411C069B049A21701A5401208646AA
:10EC7000217806980A18694601A865DF0028E9D1BD
:10EC8000694620780978401820706D1C3888A842A1
:10EC9000C1DC7046002804D020780699801B401EF5
:10ECA00088550020D6E7F8B51546069C1E4607464F
:10ECB00002220094FFF7A6FF002806D13346102257
:10ECC000294638460094FFF79DFFF8BDF7B582B09E
:10ECD00000260546167000681446002805D0284610
:10ECE000039900F0DFF806002DD1687900281BD0C9
:10ECF0002078039F001D1F2824D8684679DF00284C
:10ED000021D121780322481C20707A5421781922BD
:10ED1000481C20707A542078C1196846008800F099
:10ED2000BCF82178401820702989002923D00120BF
:10ED30008446EA680398002A07D0227853189B1C5F
:10ED40001F2B04D90C2005B0F0BD0720FBE71346AC
:10ED5000521C491C2270C15422786746511C2170F4
:10ED6000875423782A891818E96800F0DDFC207898
:10ED7000297A401820702869002815D000214156B2
:10ED800022788C46D01C03991F28DBD8501C022304
:10ED900020708B5422780A23501C20708B542078CA
:10EDA0006246431C23700A54A88A002809D02846CA
:10EDB0000094062202211430039BFFF774FF060023
:10EDC000C1D1A88B002809D028460094072203212E
:10EDD0001C30039BFFF767FF0600B4D1A88C002806
:10EDE00009D028460094152214212430039BFFF7F4
:10EDF0005AFF0600A7D1E86A002805D022460399E9
:10EE000000F085F806009ED1286B002805D0224628
:10EE1000039900F0BBF8060095D13820405D00282A
:10EE200006D022462846039900F0E2F806008AD16F
:10EE3000304688E770B50D4692B000216A461170E1
:10EE400007241171002812D00189002905D0C1685A
:10EE5000002902D00978490702D4204612B070BDBB
:10EE600002A9FFF733FF0028F8D102AE00E0002628
:10EE7000002D0BD028890028EFD101AA0AA9284625
:10EE8000FFF724FF0028E9D10AAA00E00022684623
:10EE900003790178304672DFE0E70870000A4870B5
:10EEA00002207047F8B514780746A01C15460E4698
:10EEB0001F2803D83879801C1F2801D90C20F8BDE1
:10EEC0001D20001B80B26946864608803019801CD0
:10EED0007DDF0028F3D13868022805D16846008814
:10EEE000704501D8092107E038790821002801D0B0
:10EEF000704501D968460088421C3255641CE2B254
:10EF0000B1542978801C081828700020F8BDF8B585
:10EF10000D4611780646881D14461F2801D90C207D
:10EF2000F8BD33880720062BFAD31927FF01BB420F
:10EF300002D94E4A9342F3D17288062AF0D3BA42DC
:10EF400002D94A4FBA42EBD1484FBB4203D0BA4232
:10EF500001D09342E4D8481C052220706A542078DE
:10EF60001222411C21702A54207841193088FFF761
:10EF700094FF21784018C0B2207041197088FFF7C3
:10EF80008CFF2178401820700020F8BD70B5054630
:10EF900000790E46801C1446C0B21178821C8A1873
:10EFA0001F2A01D90C2070BD0A46491C401C217043
:10EFB000B0542078FF22411C2170325420788119EE
:10EFC0002888FFF76AFF21784018C0B22070AA880D
:10EFD000002A09D0A968002908D0801900F0A4FBF4
:10EFE0002078297940182070002070BD072070BD5E
:10EFF000F7B582B002981446406B0F46002832D015
:10F00000029800252030009028E00298416B0C20E7
:10F0100068430E18217830794A1CC01C227078543D
:10F0200021781622481C20707A542078C119308823
:10F03000FFF733FF21784018C0B22070B288002A51
:10F0400009D0B16800290ED0C01900F06DFB2078FE
:10F050003179401820706D1C0098EDB2007EA842F6
:10F06000D3D800206FE607206DE60000FFFF000008
:10F0700008280CD004DC002807D006280FD108E0AF
:10F080000B280AD00C280AD105E001207047022085
:10F0900070470320704704207047042901D00620E0
:10F0A00070470520704710B50B46022819D0032879
:10F0B00016D100290BD0F748F749808888420FD035
:10F0C000132176DF00280BD0F4A29F2106E0104622
:10F0D000FEF77BF9002803D0F0A2A521FDF724F963
:10F0E00010BD01211846FFF7C3FF02460121F54874
:10F0F000FDF71CFF0028F3D0E8A2B021EEE710B521
:10F100000A46044603211046FFF7B2FF02460321D8
:10F110002046FDF70BFF002803D0E0A2CA21FDF72F
:10F1200003F910BD30B5054687B00020009001906E
:10F1300002900390D7486A46C0781070E24A10687F
:10F140009268049068460692059008790C2825D0AC
:10F15000042809D0032201212846FDF7E7FE0028F4
:10F160001AD0CEA2E82115E0886800F051FA039089
:10F1700004A8FDF7E4FC00280ED00121FFF778FF7A
:10F18000024601212846FDF7D1FE002804D0FF21C8
:10F19000C2A20931FDF7C8F807B030BD8C6820461F
:10F1A00000F036FA0190201D00F032FA029020465D
:10F1B0000830DAE7F0B5054608790E4685B08107D4
:10F1C0000AD0032211462846FDF7B0FE00281FD0C2
:10F1D000FF21B2A24F3143E0AE4900901431FEF757
:10F1E000CDF8010011D1AB4CB168009A606900F014
:10F1F0009BFA0098FEF71DF9010006D120466946EA
:10F200001430FEF722F9010004D02846FFF777FFFB
:10F2100005B0F0BD0320019000988008029060695D
:10F22000039001A8FDF7D8FC07000BD0092F1AD0D6
:10F230006069FEF7CAF8010002D02846FFF75FFFB9
:10F240003946E2E730792169012240182061032123
:10F250002846FDF76BFE0028DAD0FF218FA27F3110
:10F26000FDF762F8D4E730792169411821616078AF
:10F270000028CDD02089401E0004000C2081C7D179
:10F280002846FDF792FF002804D0FF2183A2903189
:10F29000FDF74AF8E0882081BAE710B5FF217FA288
:10F2A000CB31FDF741F810BD10B57A4C7A49A088F2
:10F2B000884208D0132176DF002811D077A2834935
:10F2C000FDF732F80CE0A078002809D074DF0028A0
:10F2D00004D07E4971A2FA39FDF726F80020A0700B
:10F2E000FFF7E1FB002804D078496CA20931FDF753
:10F2F0001BF8002010BD70B50D6804460120654A5A
:10F300002B0000F064FB0A2F393B0616234F543EB6
:10F310005822FDF7E4FC0421FFF7AAFE024604216F
:10F320002046FDF703FE00280FD0FF215BA2FD3130
:10F330004AE0FFF7B9FF002803D058A26449FCF760
:10F34000F3FFFDF7F1FC002809D170BDFFF7ACFF1A
:10F35000002804D05E4951A20D31FCF7E5FFFDF70E
:10F36000F8FC70BDD0600879002803D08868007868
:10F37000D07070BD0420FBE7022000E00320D060C5
:10F3800070BDD2682046012A06D0022A07D0032A7F
:10F39000F6D1FFF70FFF70BDFFF7C4FE70BD00F0A0
:10F3A00041F970BD50708888D080108170BD0020F8
:10F3B0005070D08070BD20461169FDF7BFFE002857
:10F3C000F8D0472135A2C900FCF7AEFF70BD10B5DB
:10F3D000304CA07800280BD13A48143873DF00284D
:10F3E00004D03B492DA24A31FCF79EFF0120A070BA
:10F3F00010BD70B5274C0588A388132D29D00ADCD1
:10F40000344A3549102D18D0112D15D1CA602078F5
:10F41000002818D019E0522D26D0552D0CD1807916
:10F42000002809D11321184676DF002804D0284986
:10F430001AA28C31FCF778FF70BD8A608088A080AA
:10F440000020A07070BDFFF7C2FF0020C043A08065
:10F4500070BD104A1846183200217FDF0028F7D00F
:10F460001B490EA28431E5E7002211461846A9DFA8
:10F470000028EDD0164909A29231DBE710B5044609
:10F48000FFF742FB21460F48FDF71EFE2046FFF71F
:10F49000B0FF10BDDC200020FFFF00002E2E5C62BC
:10F4A0006F6F746C6F616465725F6466755C6466CF
:10F4B000755F7472616E73706F72745F626C652ECB
:10F4C00063000000D427002044FA03005503000025
:10F4D00001020000000040000005005010B594B08B
:10F4E000062069460872684671DF002803D0804A0A
:10F4F0008049FCF719FF69464878401C4870002095
:10F5000070DF002804D01721794A4901FCF70CFF6D
:10F510007948694600798873784888813C2105A834
:10F5200000F061F902200590002469464C76012024
:10F53000888302A908916946088503A80B90214693
:10F5400005A8FFF777FC002804D06A49684A1831FB
:10F55000FCF7EAFE68481421143800F044F96648C4
:10F56000143804704460047233210182448214B060
:10F570008FE7604910B55E4A2E31FCF7D5FE88E76B
:10F5800010B55F4888B00024C4605E48FEF7E3FD14
:10F5900000283BD15C48FDF7CFFAFDF7C9FE0028F3
:10F5A00034D100F06FF859480090594801906946ED
:10F5B0005148FDF74FFD002804D0C7214C4A89006F
:10F5C000FCF7B2FEFFF78AFF1C21684600F00BF93A
:10F5D0005048019001208003029000940321684666
:10F5E0000173C481012101744B480690059468465B
:10F5F000FFF735FA002804D0FF213D4AE231FCF73D
:10F6000093FE00F063F8FFF7E2FE002008B040E749
:10F6100010B5044600F0E9F80002E178000A090696
:10F62000084336E7FEB50446012000908868029042
:10F630000879002283070ED08007800F0422121A57
:10F640000020034605E00E79029D3618B600AB5146
:10F65000401C9042F7D308798018800801906846D2
:10F66000FDF7F0FA0221FFF703FD024602212046D2
:10F67000FDF75CFC002804D0FF211D4A3B31FCF75C
:10F6800053FEFEBD0EB5112069460872082223A163
:10F6900002A87CDF002804D01649154A1E39FCF761
:10F6A00043FE002000900C216A4601901180FF214A
:10F6B000913151809080D18068467ADF002804D053
:10F6C0000C490B4A1439FCF72FFE0EBD0C491E20C5
:10F6D00018310880887801221043E12210400C3054
:10F6E000DF22104088700720C87010200871704712
:10F6F0009CF40300DB020000D4270020301500003A
:10F70000DC2000207DF40300A7F00300F7F20300E3
:10F7100073F50300CD0C00009BF2030049352B2D3F
:10F720004446553300000000F8B5042A2CD3830763
:10F7300012D00B78491C0370401C521E83070BD05B
:10F740000B78491C0370401C521E830704D00B78B1
:10F75000491C0370401C521E8B079B0F05D0C91A11
:10F76000DF002023DE1B08C90AE0FCF749FDF8BDD5
:10F770001D4608C9FD401C46B4402C4310C0121F52
:10F78000042AF5D2F308C91A521EF0D40B78491C8A
:10F790000370401C521EEAD40B78491C0370401CB5
:10F7A000521EE4D409780170F8BD01E004C0091FBD
:10F7B0000429FBD28B0701D50280801CC90700D029
:10F7C0000270704700290BD0C30702D00270401CA2
:10F7D000491E022904D3830702D50280801C891E9A
:10F7E000E3E70022EEE70022DFE70378C27819465C
:10F7F000437812061B0219438378C0781B0419430F
:10F8000011430902090A0006084370470022030950
:10F810008B422CD3030A8B4211D300239C464EE02B
:10F8200003460B433CD4002243088B4231D30309E7
:10F830008B421CD3030A8B4201D394463FE0C30999
:10F840008B4201D3CB01C01A524183098B4201D3B1
:10F850008B01C01A524143098B4201D34B01C01A9C
:10F86000524103098B4201D30B01C01A5241C30814
:10F870008B4201D3CB00C01A524183088B4201D383
:10F880008B00C01A524143088B4201D34B00C01A6F
:10F890005241411A00D201465241104670475DE084
:10F8A000CA0F00D04942031000D340425340002207
:10F8B0009C4603098B422DD3030A8B4212D3FC22B0
:10F8C000890112BA030A8B420CD3890192118B422F
:10F8D00008D3890192118B4204D389013AD0921145
:10F8E00000E08909C3098B4201D3CB01C01A524100
:10F8F00083098B4201D38B01C01A524143098B42C9
:10F9000001D34B01C01A524103098B4201D30B01B1
:10F91000C01A5241C3088B4201D3CB00C01A5241D6
:10F9200083088B4201D38B00C01A5241D9D24308BD
:10F930008B4201D34B00C01A5241411A00D20146FA
:10F94000634652415B10104601D34042002B00D564
:10F950004942704763465B1000D3404201B5002026
:10F96000C046C04602BD704770477047754600F0FC
:10F9700023F8AE46050069465346C008C0008546D8
:10F9800018B020B5FCF7BCFC60BC00274908B6469F
:10F990000026C0C5C0C5C0C5C0C5C0C5C0C5C0C59E
:10F9A000C0C5403D49008D4670470446C046C0462C
:10F9B0002046FCF7D2FB000000487047FC270020DF
:10F9C00001491820ABBEFEE726000200704730B4A4
:10F9D0007446641E2578641CAB4200D21D46635DEC
:10F9E0005B00E31830BC1847020000000000000074
:10F9F0000000000000000000020000000000000005
:10FA000000000000000000000000000000000000F6
:10FA100004000000000000000000000000000000E2
:10FA200000000000000000008DC80300000000007E
:10FA30000000000023D1BCEA5F782315DEEF12122C
:10FA400000000000020000000000000000000000B4
:10FA500070FA030000200020FC00000004C1030035
:10FA60006CFB0300FC2000206413000020C1030095
:10FA70000024F4000000000000000000000000006E
:10FA80000000000000000000000000000000000076
:10FA90000000000000000000000000000000000066
:10FAA0000000000000000000000000000000000056
:10FAB0000000000000000000000000000000000046
:10FAC0000000000000000000000000000000000036
:10FAD0000000000000000000000000000000000026
:10FAE0000000000000000000000000000000000016
:10FAF0000000000000000000000000000000000006
:10FB000000000000000000000000000000000000F5
:10FB100000000000000000000000000000000000E5
:10FB200000000000000000000000000000000000D5
:10FB300000000000000000000000000000000000C5
:10FB400000000000000000000000000000000000B5
:10FB5000FFFF0000000000000000000000000000A7
:10FB6000000000000000000000000000FFFFFFFF99
:10FB7000FFFFFFFFFFFFFFFFFFFFFFFFFFFFFFFF95
:10FB8000FFFFFFFFFFFFFFFFFFFFFFFFFFFFFFFF85
:10FB9000FFFFFFFFFFFFFFFFFFFFFFFFFFFFFFFF75
:10FBA000FFFFFFFFFFFFFFFFFFFFFFFFFFFFFFFF65
:10FBB000FFFFFFFFFFFFFFFFFFFFFFFFFFFFFFFF55
:10FBC000FFFFFFFFFFFFFFFFFFFFFFFFFFFFFFFF45
:10FBD000FFFFFFFFFFFFFFFFFFFFFFFFFFFFFFFF35
:10FBE000FFFFFFFFFFFFFFFFFFFFFFFFFFFFFFFF25
:10FBF000FFFFFFFFFFFFFFFFFFFFFFFFFFFFFFFF15
:08FC00000100000000000000FB
:00000001FF
